:1000000093C0ABC0AAC0A9C0A8C0A7C0A6C0A5C0C5
:10001000A4C0A3C0A2C0A1C0A0C09FC09EC006062D
:100020000707070809090A0B0C0E0F1113151719FA
:100030001C1F2225292D31353A3F44494F555C6319
:100040006A727A828B949DA7B2BCC8D3E0ECF9FFA8
:10005000FFFFFFFFFFFFFFFFFFFFFFFFFFFFFFFFB0
:10006000FFFFFFFFFFFFFFFFFFFFFFFFFFFFFFFFA0
:10007000FFFFFFFFFFFFFFFFFFFFFFFFFFFFFFFF90
:10008000FFFFFFFFFFFFFFFFFFFFFFFFFFFFFFFF80
:10009000FFFFFFFFFFFFFFFFFFFFFFFFFF0000006D
:1000A0000000000000000000000000000000000050
:1000B0000000000000000000000000000000000040
:1000C0000000000000000000000000000000000030
:1000D000010204050607090A0C0D0E10121315176C
:1000E000191A1C1E20222427292B2D303235373A8D
:1000F0003D3F4245484B4E5154585B5E6265696DC9
:100100007074787C8084888D91959A9EA3A8ADB1F7
:10011000B6BBC1C6CBD1D6DCE1E7EDF3F9FF7F8DED
:10012000969FA4A8ADB2B6FF11241FBECFEDCDBFE0
:1001300010E0A0E6B0E0E8EDF7E002C005900D9217
:10014000AC36B107D9F720E0ACE6B0E001C01D92B3
:10015000A137B207E1F720D13DC352CF20ED37E000
:10016000019720F0F9013197F1F7FACF08958AE964
:1001700092E00197F1F7089520E43FE1815020F0EB
:10018000F9013197F1F7FACF08958AEFF5CFA29AE6
:1001900081EA87B986EC86B90895369A3699FECFFA
:1001A00085B10895369A3699FECF349A84B195B1C7
:1001B000089583E5E1CF80916F008823F1F080916D
:1001C0006E006FEF90E0F8D280916E008F5F8093A9
:1001D0006E006FEF90E0F0D280916E008F5F8F73B2
:1001E00080936E006091740090E0E6D280916E0082
:1001F00090E0609173000196DFC20895DCDF6091AA
:100200006F0081E490E0D8D260916B0082E490E0CE
:10021000D3C20F931F93CF9381E490E0C5D2823075
:1002200018F480936F0002C010926F0082E490E097
:10023000BBD29FEF980F953410F480936B0010920F
:100240006E00C0916E00C034A0F40C2F10E0C80105
:10025000ABD28F3F51F080936C00C8010196A4D2BD
:100260008F3F39F080936A0004C0CE5FC0936E0068
:10027000E8CFCF911F910F9108958093700091EA7C
:100280009ABD811103C018BC19BC089590E0019774
:10029000FC01E25EFF4F2491FC01E256FF4F849186
:1002A00088BD29BD0895CF93DF93C82FD62FCC23C7
:1002B00061F080E2E2DF8D2F5FDF80E0DEDF8D2FF7
:1002C0005BDF8D2F59DFC150F2CFDF91CF910895C1
:1002D000EF92FF920F931F93CF93DF93D82FC0E23B
:1002E000E82EF12C062F10E080E8C7DFDD2319F09F
:1002F000C70134DF01C03BDF80E0BFDFC8012EDF74
:10030000C15091F7DF91CF911F910F91FF90EF9026
:1003100008951F93CF93DF938FE887B986EC86B952
:1003200041DF18E0C0E0D0E03DDFC80FD91F81E019
:1003300023DF1150C9F7CE01969587958C549440D0
:10034000DF91CF911F91089580E097DF379885B7AF
:10035000877E806185BF85B7806285BF889585B7B8
:100360008F7D85BF08951F93CF93DF93EC01862F78
:100370006FE099DF8EE300DF888111E081278883B9
:100380003DDF63E080E28FDF88811827188336DF46
:10039000DF91CF911F91F9CECF93DF93CDB7DD27BA
:1003A000CA50CDBFB99AB89A11E013BF198631DF90
:1003B0008091750081111AC0809176008F5F8F71D6
:1003C00080937600809171008F3F31F080937400AC
:1003D0008FEF809371001BC0809174008F5F8093BA
:1003E00074008A30A0F01093740011C0109276004F
:1003F00010937300109372008FEF8093710010922E
:10040000740080916F00882311F08AEF8987109221
:100410007500D1DE512CAA24A39411E0D12CE12C3B
:10042000C12CCE0101964C0128E0280F2A8767E0F5
:10043000462E480E76E4372EE2E32E2EBB24B394EC
:10044000F090740089E08F1528F0EF2DF0E0E05A6D
:10045000FF4FF0809CDE809176008031C0F095DE09
:1004600010927600B09274000FEF0093710061E07B
:100470008FE690E078DF88EF8093710062E0CE0134
:10048000099671DFB092740000937100D9CF89850D
:100490008A3F81F4198681E0F0DEB092710089DE36
:1004A00080916C008093740080916A008093730047
:1004B00082DEC6CF9DEFF91244C080917300DDDE6D
:1004C00080917600813041F48091740080937100B6
:1004D0008FEF8093720007C0823029F480917400FE
:1004E0008E5F8093710065DE8FEF80937100809145
:1004F0007600813011F48093720010927600809122
:100500007300BBDE85E038DE80917200909173004D
:1005100018161CF497FF05C008C0882311F092300C
:1005200050F0890F80937300EACF813021F480E08E
:10053000A4DE82E021DE80917200819580937200BA
:100540007BC02CEFF2120DC0AA2039F0809173000D
:1005500094DE8091730080936D002BDE1092710009
:100560006BC08EEFF8120BC0AA2029F080E885DE60
:1005700080E880936D001DDEB09271005DC097EF42
:10058000F9120CC004E080E878DE82E0F5DD80E45A
:1005900074DE8FE0F1DD0150B1F739C021EFF212C6
:1005A00011C080E86ADE81E0E7DD80E066DE8EE390
:1005B000E3DD80E862DE81E0DFDD80E05EDE8BEBA4
:1005C000DBDD3AC080EFF81203C06FE481E005C0C4
:1005D0009FEEF91204C069E280E07ADE2DC02EEEB3
:1005E000F21202C06FE0F8CF8BEFF81212C0E1DD1B
:1005F000D4DD982F80E0E82FF0E0E25EFE4FE4913A
:10060000E91710F48F5FF7CF6FE14DDEBEDDBDDD82
:1006100013C09BEEF91210C067E082E044DE05E1F2
:10062000802F2BDE5FE4752EB0DDAFDD7A94711084
:10063000FBCF0150A9F788DE10927600AEDD8F3730
:10064000F0F4C39427E02C15D8F48CEFF81621F0C1
:10065000B092740080E207C080917300823030F065
:100660008091700086958093730001C06DDE80914B
:10067000730003DE8091730080936D0086DDC12CD2
:100680009EEFF91629F08F2D8B7F883F09F089C0E6
:1006900040DE3C01111104C0DE011296F40106C0D7
:1006A000F40161922A852E13FCCFF6CF8D918193B0
:1006B0004E12FCCF688689818301081B110988EFDF
:1006C000F81225C0AA2049F020926B0080E2D5DD07
:1006D00095DD5BDD5ADD80E8D0DD33E0000F111FD2
:1006E0003A95E1F7060D171D159507951595079590
:1006F000073418F400936B0002C030926B0093E053
:10070000951510F47BDD512C54DD10E04AC094E0C7
:10071000000F111F9A95E1F7600E711E80916B001A
:1007200090E0880F991F880F991F681679061CF1B1
:1007300028E02E15E0F4681A790A830184E0159503
:1007400007958A95E1F71016110614F001E010E004
:1007500020917000822F801B803208F480E29091FB
:100760006D002132D8F09817A0F4892F12C0E394BD
:1007700010E0D12C16C08097681679066CF484E0DE
:100780008D1548F48091700090916D00891730F4B8
:100790008F5F73DD03C0D39410E002C010E0D12C52
:1007A000E12C5394A12C4CCEE199FECF1FBA8EBB05
:1007B000E09A99278DB30895262FE199FECF1CBAB0
:1007C0001FBA8EBB2DBB0FB6F894E29AE19A0FBE0A
:0807D00001960895F894FFCF93
:0C07D800FDFCFEFBEBF7F1F0EFEE013250
:00000001FF
